:04000000C6EF05F052
:0800080000C504F501C505F572
:1000100002C506F5076A03C508F50001F5C409F530
:10002000F6C40AF5F7C40BF5F8C40CF5A1AE1CEF45
:1000300000F0B1BEACEF02F009C5F5F40AC5F6F464
:100040000BC5F7F40CC5F8F404C500F505C501F5BA
:1000500006C502F5078E08C503F51100C182C180EF
:10006000C086C084C082BF9ABF98BF96BF94BF921B
:10007000BF90C19EC19CC19AC198C09AC098C196B8
:10008000C194BEEF02F0BF8ABF88BF86BF84BF8223
:10009000BF80C18EC18CC18AC188C08AC088C18618
:1000A000C1847FEF01F006013651000A00011BE018
:1000B000010A1BE0030A1BE0010A1BE0070A1BE020
:1000C000010A1BE0030A1BE0010A1BE00F0A1BE008
:1000D000010A1BE0030A1BE0010A1BE0070A1BE000
:1000E000010A1BE01CD0BF9A1AD0BF9818D0BF9647
:1000F00016D0BF9414D0BF9212D0BF9010D0C19E22
:100100000ED0C19C0CD0C19A0AD0C19808D0C09A18
:1001100006D0C09804D0C19602D0C19400D012007D
:1001200006013651000A00011BE0010A1BE0030A28
:100130001BE0010A1BE0070A1BE0010A1BE0030A9F
:100140001BE0010A1BE00F0A1BE0010A1BE0030A87
:100150001BE0010A1BE0070A1BE0010A1BE01CD0A0
:10016000BF8A1AD0BF8818D0BF8616D0BF8414D0DB
:10017000BF8212D0BF8010D0C18E0ED0C18C0CD0E7
:10018000C18A0AD0C18808D0C08A06D0C08804D0ED
:10019000C18602D0C18400D01200010E0601356F65
:1001A00033C636F600017FDF0601356B3451000A95
:1001B000000109E0010A0EE0030A13E0010A18E059
:1001C000070A1DE023D0CEB004D0010E0601356F22
:1001D00000011CD0CEB204D0010E0601356F000123
:1001E00015D0CEB404D0010E0601356F00010ED03B
:1001F000CEB604D0010E0601356F000107D0CEB88F
:1002000004D0010E0601356F000100D033C636F66A
:1002100087DF060135C601F500018EEF01F0BF9AB8
:10022000BF98BF96BF94BF92BF90C19EC19CC19A18
:10023000C198C09AC098C196C194C8EF01F0060158
:100240003351000A00010BE0010A14E0030A1EE02A
:10025000010A28E0070A32E0010A3CE047D0020127
:10026000AC9FC08CB00EAB6FAF6B8A0EAE6FAD6B38
:10027000AC8F3DD00201AC9FC08CB00EAB6F010EB5
:10028000AF6FA00EAE6FAD6BAC8F31D00201AC9FE3
:10029000C08CB00EAB6F030EAF6F400EAE6FAD6B88
:1002A000AC8F25D00201AC9FC08CB00EAB6F060E98
:1002B000AF6F820EAE6FAD6BAC8F19D00201AC9FE9
:1002C000C08C300EAB6F060EAF6F820EAE6FAD6B93
:1002D000AC8F0DD00201AC9FC08C300EAB6F0D0EF9
:1002E000AF6F040EAE6FAD6BAC8F01D00201000199
:1002F00012000601326B32C62EF60001C4D606018A
:100300002C6B2C510D0842E32D6B2D5104083CE35E
:100310002CC633F62DC634F600013FD7015231E02A
:1003200006012C39006EF00E00160050F00B316FF4
:100330002D513113036A31511D0FE96E050E032053
:10034000EA6EEFC42EF62E51800A000105E0010A84
:1003500007E0030A09E00DD006011D8F2E6B10D0B7
:1003600006011D8D2E6B0CD006011D8B2E6B08D047
:1003700000012CC62FF62DC630F62EC632F6060129
:10038000000106012D2BC1D72C2BBBD7000147D76D
:1003900032C62EF606012E53D8B495D02E517F08C2
:1003A000D8A091D01F5306E02E512F0803E1050E6F
:1003B0002E6F89D01D51400A000105E0C00A11E0EE
:1003C000E00A37E06CD006012E51600808E22E5199
:1003D0007A0805E3610E2E5D010F2E6F01D02E6BA2
:1003E00072D006012F39006EF00E00160050F00B8F
:1003F000316F305131133187036A31511D0FE96E6E
:10040000050E0320EA6EEFC42EF61E5311E02E51A6
:10041000400806E22E515A0803E3200E2E2708D08A
:100420002E51600805E22E517A0802E3200E2E5F5D
:100430004AD006012E51310A00010BE0030A0EE0FA
:10044000010A12E0070A16E0010A1AE0030A1EE098
:1004500023D01C6A1CC533F6F2DE1ED0010E1C6EC2
:100460001CC533F6ECDE18D0020E1C6E1CC533F62C
:10047000E6DE12D0030E1C6E1CC533F6E0DE0CD097
:10048000040E1C6E1CC533F6DADE06D0050E1C6E9B
:100490001CC533F6D4DE00D0060115D000010601DC
:1004A0001E5311E02E51400806E22E515A0803E374
:1004B000200E2E2708D02E51600805E22E517A0812
:1004C00002E3200E2E5F2EC601F50001BFEF02F001
:1004D000B2A2FED70201A36F000173EF02F0060182
:1004E0002C510001F5D712002CC636F619DE060194
:1004F0002D51000A000109E0010A09E0030A09E0A0
:10050000010A09E0070A09E00AD0C19208D0C190A7
:1005100006D0C09604D0C09402D0C09200D0120081
:100520002CC636F6C0DD06012D51000A000109E097
:10053000010A09E0030A09E0010A09E0070A09E0E3
:100540000AD0C18208D0C18006D0C08604D0C08441
:1005500002D0C08200D01200000103011AA901D00C
:10056000196B070E186F0601222BD8B4232B2151CB
:100570000A08D8A453D01D6B000170D5BAD601C5A6
:100580002BF606012B5318E02B517F0815E3205161
:100590002B5D12E1235100080EE2FF0A03E1225114
:1005A000F40809E22BC62CF6000199DF3C0E060187
:1005B000225F000E235B02D0236B226B2B532CE0B7
:1005C00020512B5D29E02B51850A000103E0010A2F
:1005D00011E019D006011D51800A000101E008D088
:1005E00006011E5302E01E6B02D0010E1E6F01D0E9
:1005F000060112D006011F5302E01F6B02D0010E4C
:100600001F6F0AD0000106012B51800B05E12BC69C
:100610002CF6000164DF06012BC620F6212B2151A8
:100620000B0801E1216B2151000A000105E0050AD8
:100630000DE00F0A1CE025D006011E5306E02C6BCE
:10064000020E2D6F000150DF06011CD006012C6B3D
:10065000020E2D6F000164DF06011F5307E00D0E2F
:100660002C6F040E2D6F00013FDF06010BD00D0E25
:1006700006012C6F040E2D6F000152DF060102D01F
:1006800000010601B19E00011CEF00F0060EEA6EAB
:10069000250EE96EEF500EE0140E016E006A002E7A
:1006A000FED7012EFBD7BF0E006E002EFED700D066
:1006B000EF2EF2D71200C89CC992C182C990C180A6
:1006C000C896C086C894C084C892C082C79ABF9A90
:1006D000C798BF98C796BF96C794BF94C792BF925A
:1006E000C790BF90C99EC19EC99CC19CC99AC19A1E
:1006F000C998C198C89AC09AC898C098C996C19616
:10070000C994C19420EF06F00601266B256B265193
:1007100000080BE31D0E2525E96E050E2621EA6E65
:10072000EF6A252BD8B4262BF2D7610E2F6E410E1F
:10073000376E620E0501706F420E786F630E506E59
:10074000430E586E640E4F6E440E576E650E4E6E1D
:10075000450E566E660E5F6E460E676F670E6F6FC4
:10076000470E776F680E7F6F480E876F690E9E6F1A
:10077000490EA66F6A0E8F6F4A0E976F6B0E9F6FB2
:100780004B0EA76F6C0EAF6F4C0EB76F6D0E906F68
:100790004D0E986F6E0E806F4E0E886F6F0EAE6F9F
:1007A0004F0EB66F700EBE6F500EC66F710E2E6E6E
:1007B000510E366E720E5E6E520E666F730E3F6E87
:1007C000530E476E740E6E6F540E766F750E8E6FED
:1007D000550E966F760E606F560E686F770E3E6EF2
:1007E000570E466E780E406E580E486E790E7E6F2C
:1007F000590E866F7A0E306E5A0E386E310E2D6E8F
:10080000210E356E320E3D6E400E456E330E4D6E2E
:10081000230E556E340E5D6E240E656F350E6D6FB2
:10082000250E756F360E7D6F5E0E856F370E8D6FE0
:10083000260E956F380E9D6F2A0EA56F390EAD6F7F
:10084000280EB56F300EBD6F290EC56F2D0ECD6F02
:100850005F0ED56F3D0EDD6F2B0EE56F080EED6F51
:10086000F56F5B0ECE6F7B0ED66F5D0EDE6F7D0E6D
:10087000E66F5C0EEE6F7C0EF66F3B0EBF6F3A0EAE
:10088000C76F270ECF6F220ED76F2C0EA06F3C0EB6
:10089000A86F2E0EB06F3E0EB86F2F0EC06F3F0EBA
:1008A000C86F0D0EEF6FF76F090E1E6E266E1B0ED2
:1008B0001D6E7E0E256E200E716F7E0E796F130EEB
:1008C000A16F180EB16F040EC16F810E216E850EDF
:1008D0001F6E800E206EE06F830E316E820E416EB1
:1008E000840EF16F000121EF06F00601256BD6C4DE
:1008F00026F6D69E0001446B436B380E456F416B64
:1009000040814651060126BFD68E4F0802E0010EF7
:10091000256FD6C426F6D69E0001446B010E436FA8
:10092000380E456F416B40814651060126BFD68E79
:100930004B0802E0010E256FD6C426F6D69E0001B4
:10094000446B020E436F380E456F416B4081465138
:10095000060126BFD68E490802E0010E256FD6C4D7
:1009600026F6D69E0001446B030E436F380E456F8A
:10097000416B40814651060126BFD68E520802E0E7
:10098000010E256FD6C426F6D69E0001446B040ED8
:10099000436F380E456F416B40814651060126BFBB
:1009A000D68E410802E0010E256FD6C426F6D69EEB
:1009B0000001446B050E436F380E456F416B40815B
:1009C0004651060126BFD68E4B0802E0010E256F68
:1009D000D6C426F6D69E0001446B060E436F380E31
:1009E000456F416B40814651060126BFD68E5508A2
:1009F00002E0010E256F25C601F5000122EF06F089
:100A0000D6C400F5D69E446B436B380E456F4F0E2F
:100A1000466F030E416F550E426FAA0E426F408122
:100A200040B1FED70050D612D6C400F5D69E446B16
:100A3000010E436F380E456F4B0E466F030E416F2C
:100A4000550E426FAA0E426F408140B1FED7005052
:100A5000D612D6C400F5D69E446B020E436F380EF4
:100A6000456F490E466F030E416F550E426FAA0E39
:100A7000426F408140B1FED70050D612D6C400F577
:100A8000D69E446B030E436F380E456F520E466F71
:100A9000030E416F550E426FAA0E426F408140B166
:100AA000FED70050D612D6C400F5D69E446B040E75
:100AB000436F380E456F410E466F030E416F550E62
:100AC000426FAA0E426F408140B1FED70050D6124D
:100AD000D6C400F5D69E446B050E436F380E456FA5
:100AE0004B0E466F030E416F550E426FAA0E426FBA
:100AF000408140B1FED70050D612D6C400F5D69E34
:100B0000446B060E436F380E456F550E466F030E4D
:100B1000416F550E426FAA0E426F408140B1FED721
:100B20000050D6121C6AD6C400F5D69E446B0A0E3D
:100B3000436F380E456F1CC546F0030E416F550ECE
:100B4000426FAA0E426F408140B1FED70050D612CC
:100B500025EF06F0D6C425F6D69E446B0A0E436FE9
:100B6000380E456F416B40814651060125BFD68E38
:100B70001C6E1B6AD6BE1B8ED69E1CC533F60001AA
:100B80001FEC01F01BBED68E26EF06F0F86AD69A4F
:100B9000078E0E01550E0201006FAA0E006F009124
:100BA000170E726F200E176F550E006FAA0E006F92
:100BB0000081AC9FC89CC08CB00EAB6FAF6B8A0E2F
:100BC000AE6FAD6BAC8F06011E6B1F6B0401006B2B
:100BD000086B106B186B206B0001716B726B736B81
:100BE000706B756B766B776B746B0601206B216B8A
:100BF000226B236B0001B06BAF6BB36B030EB16F55
:100C0000600EAD6F0A0E0601256F00013FDDB06B6F
:100C1000AF6BB36B050EB16F600EAD6F0A0E0601C0
:100C2000256F000133DDB06BAF6BB36B080EB16F96
:100C3000600EAD6F0A0E0601256F000127DD3BD562
:100C400063D553D60152D8A4DBD684D71CC524F66D
:100C5000800E03011A6F460E1B6F1AA901D0196B83
:100C6000070E186FA18EC00ED6121C500601245D0F
:100C700018E01CC524F6D6C400F5D69E0001446BCE
:100C80000A0E436F380E456F24C646F0030E416FBF
:100C9000550E426FAA0E426F408140B1FED7005000
:080CA000D6120301E2D70300A4
:020000040030CA
:0A0000008FFF36DF9FFFFFFFFFFFB9
:00000001FF
